:0300000002104BA0
:03000B000200A24E
:03002B000202CE00
:03005B0002041884
:030073000203F293
:1000800002030406080C10182030406080040608A3
:100090000C10182030406080A0C005050D0503033A
:1000A0000302C2AFC0D0C0E020622C20680241BA77
:1000B000306602417A302F02E4730563C3740595FC
:1000C0002540F5956340F12069EE758A78E5257045
:1000D00003758A000202C785258AC262E525F4708D
:1000E000022141206802212E207210758B00D0E081
:1000F000D0D0C283C294C295D2AF32C283C294C25E
:10010000957408D5E0FDE53C1420E21520E10D20B2
:100110007D02D297307D02D28002013ED28202015E
:100120003E207D02D280307D02D29702013E758B47
:1001300000D0E0D0D0C283C294C295D2AF32758BCA
:1001400000D0E0D0D0D2AF3241BAE525600A207DA0
:1001500002D283307D02D295C29441BAE525600275
:10016000D294207D02C295307D02C28341BAE5253A
:10017000600A207D02D295307D02D283207D02C2AA
:1001800083307D02C29541BA207D02C280307D025B
:10019000C297207D02C297307D02C2807406D5E0EE
:1001A000FDE525600A207D02D283307D02D295C212
:1001B0009441BA207D02C280307D02C297C282740F
:1001C00006D5E0FDE525600A207D02D283307D0260
:1001D000D295C29441BAC282207D02C280307D0293
:1001E000C2977406D5E0FDE5256002D294207D0219
:1001F000C295307D02C28341BAC282207D02C2977D
:10020000307D02C2807406D5E0FDE5256002D294FF
:10021000207D02C295307D02C28341BA207D02C298
:1002200097307D02C280C2827406D5E0FDE525606C
:100230000A207D02D295307D02D283207D02C283C6
:10024000307D02C29541BA207D02C297307D02C244
:1002500080207D02C280307D02C2977406D5E0FD09
:10026000E525600A207D02D295307D02D283207D73
:1002700002C283307D02C29541BA30723DE53C2016
:10028000E21A20E129207D02C280307D02C297203F
:100290007D02C297307D02C2800202BA20E1E620D0
:1002A0007D02C280307D02C297C2820202BAC2823F
:1002B000207D02C297307D02C280E525F4F58A7563
:1002C0008B00756300D262D0E0D0D0D2AF32C2AF23
:1002D000C2AD53E6EFC0D0C0E0D2D3D2AFC2CEE5BC
:1002E0002960072074461529612C78007900E58083
:1002F000307E01F430E50278FF53DACF207E0343ED
:10030000DA20307E0343DA10C2D8C271E580307E35
:1003100001F430E50279FFC3E89970CE30610375CE
:1003200029182074037529188859D270E52A6004A9
:10033000152A613C20740543DA01C2D8207002619D
:1003400097A859206102C270207431C3E894F0402C
:100350000374F0F8E8C4540F28F87984B7030261F5
:100360007CC313C3138721200802C313200A06C3CA
:10037000C898F8617C28F8500374FFF8C3E89562C8
:100380005003E562F8882230690AC3E522955E4091
:1003900003855E22852224A824C3E524955E4002BD
:1003A000A85E8825C3E52594404002D26420CF0C86
:1003B000D0E0D0D0C2D343E610D2AD32C2CF780164
:1003C000E52960053074021529C3E55994014005FB
:1003D000755C0061E6755D00756400E55C2401F5FF
:1003E0005C5003755CFFD0E0D0D0C2D343E610D29E
:1003F000AD32C0D0C0E0C2AF53917F53E67FC26040
:10040000759100C3E49550F594E49551F595759177
:1004100004D0E0D0D0D2AF32C2AF53E6EFC2ADC00D
:10042000D0C0E0C0F0D2D3D2AFA8FBA9FCC2D83074
:100430007102817F53DACF207E0343DA10307E03CE
:1004400043DA20D271E580307E01F420E502815646
:1004500088268927C1BB53DACF207E0343DA2030B8
:100460007E0343DA10C2D8C271307402C1A778008B
:0F047000E580307E01F430E502C1A78859C18EC6
:10047F0053DACF207E0343DA20307E0343DA10C2F3
:10048F0071206102A14F53DACF207E0343DA10307F
:10049F007E0343DA20C2D8D27188548955C3E895B8
:1004AF0052F8E99553F9E4FB7E027A00C3E8948C85
:1004BF00E994005005755800A13FC3E894C8E9942A
:1004CF00005008E4D2E4FB7A0AA11CC3E89468E95F
:1004DF0094015008E4D2E3FB7A0FA11CC3E894D037
:1004EF00E994025008E4D2E2FB7A1EA11CC3E894FF
:1004FF00A0E994055008E4D2E1FB7A3CA11CC3E8C3
:10050F009498E994085008E4D2E0FB7A787E00C30F
:10051F00E89556FCE99557FD30E708ECF42401FC0B
:10052F00EDF4FD755800C3EC9AED9E50037558011C
:10053F0088568957A854A955885289537802C18E75
:10054F00C3E89526F8E99527F9307C02C172307B14
:10055F0002C172307A02C16B207502A172E9FDE807
:10056F00FCA191E9C313F9E813F8307902C16BE9E3
:10057F00C313F9E813F8307802C16BE9C313FDE830
:10058F0013FC206126C3EC941CED94024002A1A839
:10059F00ED7018C3EC94C850120528C3E528940ACF
:1005AF005002C1A7755900D270C1A7E52860021586
:1005BF00287400207F0B7888E67896B40302789E23
:1005CF00E624FAFEE43400FFC3EC9EFCED9FFD929F
:1005DF00087888E6B40327A2085009207D20C2AF0F
:1005EF00D27DA1FA307D17C2AFC27DC283C294C241
:1005FF0095C280C282C297206902D26BD2AFA20885
:10060F005017E6B4030DECF42401FCEDF43400FDB7
:10061F0002062878007900C1727888E6B40315ECD9
:10062F0033FCED33FDC3EC940AFCED9400FD500454
:10063F007C007D00C3EC94FFED9400400678FF79B9
:10064F0000C172EC856FF0A4C5F0A2F733F8790002
:10065F00400302068E78FF790002068EE9C313F974
:10066F00E813F8307C0EE9600278FFC3E81338F81E
:10067F00E43400F9C3E894FFE99400400278FF885E
:10068F0059D270206102C1A7741FF4552F4BF52F5B
:10069F00C274E42B7002D274752918307403752953
:1006AF000A306102C1BB20740353DAFE752A06308B
:1006BF007403752A0AD0F0D0E0D0D0C2D3D2AD43A4
:1006CF00E6103279010206F079030206F0790A0288
:1006DF0006F0791E0206F079640206F079C8020668
:1006EF00F07817E4D5E0FDD8FAD9F6227A147B78A2
:1006FF000207177A107B8C0207177A0D7BB402075B
:10070F00177A0B7BC8020717AC257525017902B242
:10071F007DE4C282D5E0FDE5256002D294D5E0FDEF
:10072F00C294D5E0FDD282D5E0FDE525600A207D9B
:10073F0002D283307D02D295E570D5E0FD207D0297
:10074F00C283307D02C2957496D5E0FDD9C1EAF817
:10075F00D5E0FDD8FBDBB1C2828C2522C37C007DA6
:10076F000075F00005F0EA33FAEB33FB50F6EB13AC
:10077F00FBEA13FAC3E9FFE8FEE89AF8E99BF950A0
:10078F0004EFF9EEF8B3EC33FCED33FDD5F0DFED0C
:10079F00F9ECF822E889F08A20D2D4F8A9F07B008E
:1007AF0030F70B7BFFF42401F8E9F43400F9E88506
:1007BF0020F0A4ADF0F8E98520F0A4AFF0FEED2E07
:1007CF00F974003FFA7C04C3EA13FAE913F9E8134A
:1007DF00F8DCF48BF030F70AE8F42401F8E9F4348C
:1007EF0000F9E889F0C2D4F8A9F02222E547603B6E
:1007FF00C3E53B13F9E53A13F8C3E53E98F8E53F37
:10080F0099F9500CC3E89480E994FF40160208361A
:10081F00C3E8947FE994005003020836787F79008B
:10082F00020836788079FF8843894422E54760586B
:10083F00E5432540F8E5443541F9854420E4300788
:10084F0001F43542FA30E709C3EA94F04015020883
:10085F0078C3EA940F500302087878FF79FF7A0F74
:0E086F00020878780079007AF0C3E524955EDF
:10087D005006E52460090191E54420E70D0191E55D
:10088D004430E706884089418A4222E547700302D9
:10089D0008FC78A1E6FAC3E54333F8E54433F912D1
:1008AD0007A3E930E70BC3E89480E994FF401301F7
:1008BD00D3C3E8947FE99400500201D3787F790087
:1008CD0001D3788079FFE820E715C3E52398F84038
:1008DD0009C3E8940140030208FA78010208FAE816
:1008ED00F424012523F840030208FA78FF884522F5
:1008FD00E547700302095F78A2E6FAA841A9421202
:10090D0007A3E930E70CC3E89401E994FF40160210
:10091D000936C3E894FFE99400500302093678FFC5
:10092D007900020936780179FFE920E715C3E5451D
:10093D0098F84009C3E89401400302095D7800026C
:10094D00095DE8F424012545F8400302095D78FFAF
:10095D0088242278FFC264E52D5406702FD264C31B
:10096D00E53B940A4009C3E52594405002C264E575
:10097D003B601974FF853BF0848537F0A4F8C5F012
:10098D00600278FFC3E895615002A8618860220279
:10099D000A397883E6F520120E6375E8901206D2B7
:1009AD0075E890E5E820ECFBA8BDA9BE120EF9751F
:1009BD006B55756C00C3740013FD745513FC7455A1
:1009CD002CFC74003DFDECFAEDFBC3E89AE99B406D
:1009DD0014E56B2455F56BE56C3400F56CEA2CFAD7
:1009ED00EB3DFB80E5AE6BAF6CC3E56C13F9E56BCE
:1009FD0013F8C3E913F9E813F8E56B28F569E56C0D
:100A0D0039F56A7A03C3E913F9E813F8DAF7AA207E
:100A1D001A7009756B00756C00020A391AEA6008C4
:100A2D00EE28FEEF39FFDAF88E6B8F6C2275E890A9
:100A3D00227883E6FFE5E820ECF7A8BDA9BE056D99
:100A4D00C3E56D94084052756D00E9FA79A0E76031
:100A5D0044EA7007E56E601B020A74C3E8956E6088
:100A6D0010E56E5006600C14020A800460F9020A4B
:100A7D0080E56EF56EC3946D401B755EC0C3940426
:100A8D004013755E80C39404400B755E40C394049F
:100A9D004003755E0075BB0922E55EF46002055EDC
:100AAD00E56DB4070375BB1022743279A387F0A4EA
:100ABD00C5F0A2F733F8C3E8955E4002A85E882220
:100ACD0088248825886122753A00753B7F2275C878
:100ADD0020A8CCA9CD75C824AA38AB398838893956
:100AED00C3E89AF8E99BF9AA3AAB3BAC3AAD3B7E29
:100AFD00047F02C3EB940440021E1FC3EB94084015
:100B0D00021E1FC3ED13FDEC13FCDEF7C3EA9CFAC6
:100B1D00EB9DFBEF6009C3E913F9E813F8DFF7EA82
:100B2D0028FAEB39FB8A3A8B3B400122753AFF7567
:100B3D003BFF223060026140854C50854D51D260A3
:100B4D0043E680227892E6FFC3E535948240010F9B
:100B5D00C3E53594A040010FC3EF940640027F0515
:100B6D007E021E3072010EC3E53B940350060E0E3D
:100B7D003072010EC3E53B940250060E0E30720129
:100B8D000EA93BA83A7A04C3E913F9E813F8DAF78A
:100B9D00C3E89EF8E99400F94009C3E89402E9948A
:100BAD000050047802E4F9E9FBE8FAC3E913FDE823
:100BBD0013FC884C894DC3EF94036037EF20E00D93
:100BCD00E82CF8E93DF9ECFAEDFB020BEDE828F81D
:100BDD00E939F9C3E89402F8E99400F97A02E4FBE3
:100BED00C3EF9403400D8A4E8B4F884889498C4A38
:100BFD008D4B22884E894F8A488B498C4A8D4B22CA
:100C0D00306002810DD26043E680E52D54066027E9
:100C1D00A83AA93BE53494085006E820E002A94D16
:100C2D00759100C3E498F594E499F595759104D206
:100C3D006053917F43E68022D265753D007520009B
:100C4D00020C58D265753D00752040E52D540660A7
:100C5D0002C265D2AF206005E53D60012278017AC0
:0F0C6D0002C3E53B940540027802C3E53B940ABD
:100C7C0040027803C3E53B940F40027A03306904C9
:100C8C00781E7A01206007E53D6003D2AF22D2AF17
:100C9C000000C2AFC3E53BFB940F40027B0FEB049B
:100CAC003073012320620123F93069027982E58BCC
:100CBC00C39940D0053DEAFBE59BF45440B52004B4
:100CCC00DBF681F42065028158C265759100AE3A5D
:100CDC00AF3BC3E49EF594E49FF595759104D26007
:100CEC0053917F43E68081583065028158D895D264
:100CFC00AF2230690B0534206016753400020D1CD0
:100D0C0020600D20650A206B071581158102151BCB
:100D1C0022A84EA94F75910053917FC3E498F59486
:100D2C00E499F595759104854850854951D26043F5
:100D3C00E6802278003064053065027801E535756F
:100D4C00F007A4F9E5F028F5F0E9A2F013A2F113ED
:100D5C00A2F213F535C394785003753578C3E53595
:100D6C0095364008D266C283C294C295306002A107
:100D7C0078854A50854B51D26043E68022C2AFC27F
:100D8C0080C282C29730720B90021C7406D5E0FDB3
:100D9C00020D9F207D02D280307D02D297759F4339
:100DAC00753C02020EDEC2AF207D02C295307D0280
:100DBC00C2833072179001F9C282207D02C2973033
:100DCC007D02C2807406D5E0FD020DDB90015C3023
:100DDC006206E5256002D294207D03759F53307D19
:100DEC0003759F33753C03020EDEC2AFC280C28214
:100DFC00C29730720B9001D67406D5E0FD020E0C32
:100E0C00207D02D297307D02D280207D03759F33E6
:100E1C00307D03759F53753C04020EDEC2AFC29445
:100E2C003072179001B3207D02C280307D02C297D0
:100E3C00C2827406D5E0FD020E4990014A30620E62
:100E4C00E525600A207D02D283307D02D295759F04
:100E5C0043753C05020EDEC2AFC280C282C297301F
:100E6C00720B9001887406D5E0FD020E79D28220B7
:100E7C007D03759F53307D03759F33753C06020EC1
:100E8C00DEC2AF207D02C283307D02C29530721F5C
:100E9C00900247207D02C280307D02C297207D02E5
:100EAC00C297307D02C2807406D5E0FD020EBE9062
:100EBC00016E30620EE525600A207D02D295307DF0
:100ECC0002D283207D03759F33307D03759F53754C
:100EDC003C01306B13120EF97406D5E0FD7408D585
:100EEC00E0FDD280D282D297C266D2AF2290014866
:100EFC00C283C294C295C280C282C297C262227857
:100F0C008076FF0876FF0876FF0876FF08760308E0
:100F1C007604087609087603087601087601788C41
:100F2C0076010876FF0876FF0876FF0876FF0876CC
:100F3C00FF0876030876FF0876FF0876FF0876250B
:100F4C000876D00876FA0876FA0876040876FF0850
:100F5C00760108760008767A0876FF087601227802
:100F6C0087E6FFC272BF0302D2727888E6C394038D
:100F7C006008C27DE630E102D27DC27E7889E6301F
:100F8C00E102D27EC3EF94026008758E01D2730227
:100F9C000FA3758E00C273227880E61490008093A4
:100FAC0078A1F67881E6149000809378A2F6D1F9B6
:100FBC00227886E61490008D9378A3F6D1F922223C
:100FCC00789CE67536FF75370CB402067536A0753D
:100FDC00370AB4030675368275370522D281789D9F
:100FEC00E66002C281227896E6FA7897E6FB307FBB
:100FFC00047A007BFFC3EB9AFCC3948250027C8280
:10100C00756F00056FEC856FF0A4C3E5F09480401C
:10101C00F222D27F120FF21206E17A007B007C10D2
:10102C001206D7E5592AFA74003BFBDCF37C04C3A7
:10103C00EB13FBEA13FADCF7FEC27F120FF222E588
:10104C00EF20E6037520000520903FFFE52014609B
:10105C0006901DFF1460009304600375EF12C2D359
:0F106C0053D9BF7581C043FF801206D275EF02C2
:10107B0043B203E5B3240420E702F5B3120EF9756E
:10108B0080F075A40F75F13F75D4DF75904F75A582
:10109B00B075F2F575D50075A60175E241120F0B0F
:1010AB0012154D78988670C2AF1206EB1206FB1222
:1010BB0006E11207021206E11207091206E11216E7
:1010CB00611206EB1206EB1206E6C2AFE4F8F6D895
:1010DB00FD78C879C8308507D9FBD8F7021C0012F8
:1010EB000F0B12154D120F6B120FA4120FBD120F17
:1010FB00CB120FCC120FE8120FF278988670120EEB
:10110B00F975885075891275C82475910475D84086
:10111B0075A82275B80275E690759B80759D007554
:10112B00D10E75BC5875BB0975BA1175E8801206DE
:10113B00D2D2AF12099C43DA01C2D8C2711206EBAC
:10114B00753001D2617B037A0CE55870067A0CDBA3
:10115B000201D51206E120700201D5C270E559C318
:10116B00940240E3E52F541F855B5AF55BB55AD7C4
:10117B00DAD7C26153DACF207E0343DA20307E0305
:10118B0043DA10C2D8C271C2757528001206E63058
:10119B007409C3E528940A4002D2751206D7780267
:1011AB003074027800C3E5599840F0C2AF1206FBC9
:1011BB001206FB1206FBD2AF1206EB7546007888BF
:1011CB00E6B4030241AA1206D7788CE6C394015009
:1011DB00030212AAE530C3940150030212AA207431
:1011EB0035C3E55994FF50030212AAC2AF12071080
:1011FB00D2AF1206E6C3E559940150EFC2AF120607
:10120B00FB1206DC1206FBD2AF1206E6C3E55994BD
:10121B00FF40E90216E67F05D27F120FF21206E6B7
:10122B00C2AFC27F120FF2AE59C3E559947FD2AF52
:10123B0040771206D2C2AF120710D2AFDFDA111EFF
:10124B00C3EE94057897F61206EB12158F121669FA
:10125B007F0AD27F120FF21206E6C2AFC27F120FC5
:10126B00F2AE59C3E559947FD2AF50E41206D2C205
:10127B00AF1206FB1206DC1206FBD2AFDFD4111E37
:10128B00EE24057896F61206EB12158F12169812AD
:10129B0006E6120FF2C3E55994FF40F30216E6C3BC
:1012AB00E559954640038559461206E6780179883B
:1012BB00E7B403027805C3E55998400221C9C2AFD0
:1012CB00120710120710120710D2AF1206EB75306F
:1012DB0000E4F531F5320531E531F470390532783A
:1012EB009AE67819146012783214600D787D1460C8
:1012FB000878FA146003753200C3E532984017156D
:10130B00327531B478998670C2AF120710D2AF78AC
:10131B009886701206E61206DCE529700530740219
:10132B0001D578012074027806C3E5599840A77857
:10133B0088E6C3940360031206E6E529700201D523
:10134B00C2AF120EF9E4F522F523F524F525D2AF41
:10135B0078858662F53EF53FF540F541F542F56D32
:10136B00F547F52CF52DF535120AD4756D0875BBBF
:10137B00101206D2120A3AE5E820ECFBA8BDA9BE72
:10138B00E97001F8886E120A3E756D0875BB10780E
:10139B0087E6FE7602120F6B7887EEF6C2AF755EAC
:1013AB00FF120AB685225E85225F852260D2AF7559
:1013BB002201752401752501855D64756501D2686F
:1013CB00D269753400120E63120E8D120AD4120AF2
:1013DB00DB120B510213EE120EF9120F6B756D002F
:1013EB0075BB09120C50120CFE120D1D1207FA12CE
:1013FB000D3F120D89120ADB120B40120B51120C0E
:10140B000D120C45120CFE120D1D1207FB1209607A
:10141B00120D3F120DB2120ADB120B40120B5112BE
:10142B000C0D120C50120CFE120D1D12083B120D5E
:10143B003F120DF6120ADB120B40120B51120C0D60
:10144B00120C45120CFE120D1D120898120D3F12B4
:10145B000E28120ADB120B40120B51120C0D120C40
:0D146B0050120CFE120D1D1208FD120D3F57
:10147800120E63120ADB120B40120B51120C0D12E2
:101488000C45120A3A120CFE120D1D120A3E120DDC
:101498003F120E8D120ADB120B40120B51120C0D6B
:1014A800306935206B3285615E85615F855D647565
:1014B800650179327A0AC3E53499400FC269D26A64
:1014C8008A33755EFF755FFF0214E0C3E559940126
:1014D80040030213EE02151B306A1B206B18E5331C
:1014E800147004C26A61E2F533C3E55994014003FC
:1014F8000213EE02151BC3E55C9482501630740487
:10150800E529600FC3E53B78F0306B0278609850AE
:101518000261EEC2AF120EF97887E6FE7602120F6C
:101528006B7887EEF6E4F522F523F524F525F562C8
:10153800C268D2AF1206D2120EF9307406E52970CD
:101548000201D541DC901A0D78201215D1E520B49E
:101558005A0CA31215D1E520B4A50302156F120F7A
:101568000B12158F02158E901A0378807B0A1215BC
:10157800D1A308DBF9901A0F788C7B151215D1A32B
:1015880008DBF9901A2422C2AF1216101215EA903D
:101598001A00740D1215D6A374021215D6A374136B
:1015A8001215D6901A0378807B0A1215D5A308DB8A
:1015B800F9901A0F788C7B151215D5A308DBF91250
:1015C8001623121601901A2422E493F622E6438F7A
:1015D80001538FFD75EF0275B7A575B7F1F0538FFD
:1015E800FE22438F02438F0175EF0275B7A575B7C9
:1015F800F1901A0DF0538FFC22901A0D745AB1D63F
:10160800901A0E74A5B1D6227A3079D07820901A23
:1016180040B1D1E520F709A3DAF7227A3079D090E2
:101628001A40E7B1D609A3DAF922AB71A872BB0157
:10163800027984BB02027985BB03027986BB040266
:101648007992BB05027987BB0602799CBB070279B0
:1016580088BB08027989E8F7227C051206EBDCFBD7
:1016680022C2AF1206FB1207021207091207101254
:1016780006DC1206FB1207021207091207101206EF
:10168800DC1206FB120702120709120710D2AF225A
:10169800C2AF1207101207091207021206FB120640
:1016A800DC1207101207091207021206FB1206DCE9
:1016B8001207101207091207021206FBD2AF22AE58
:1016C80071AF72C2AF1206FB1206FB1206FB1206BE
:1016D800DCDEF21207101206DCDFF8D2AF22D16985
:1016E800D161D161757101757201757300D1C77CC3
:1016F80005AD591206EBC3ED955970F5C3E559943C
:1017080001400AC3E55994FF4032021722D132B191
:101718008FD169C2AF75EF12D161DCD50573C3E50E
:10172800739403500280C6D1610572E5711490006C
:101738009A93F808C3E57298500280AED161D161DE
:101748000571C3E57194095002809C120F0BB18F8B
:07175800C2AF75EF12D16171
:101A00000D0213FFFFFFFF0304090301015AA501A3
:101A1000FFFFFFFFFF03FFFFFF25D0FAFA04FF01DE
:051A2000007AFF01FF48
:101A400023416C69676E424C33355023202020209F
:101A500023424C48454C4923463333302320202031
:101A60002020202020202020202020202020202076
:101C0000C2AFC2D353D9BF7581C043B20343FF8073
:101C1000752438752503B1BF75EF0275E24043F1B5
:101C20002053A4DFD285780379E67C1075220075F5
:101C30002300901DCC7B0675249875250130850204
:101C4000813D208508D8FBD9F9DCF781AD308508C6
:101C5000D8FBD9F9DCF781ADB17FE493A3C39A60D7
:101C6000028126DBDDB171600281267B08E493FAF4
:101C7000A3B152DBF87A30B152752200752300B15E
:101C800071EAFCEBFDC3ED94FE400EB1718A278B27
:101C900028ED30E0048A828B83B1717AC270D8C398
:101CA000ED94FE601050CEBD0022EC600675200061
:101CB0000200008100A827A9280809D804D90281B8
:101CC000C9B175EA89AAF281BB0D8199C3ED94036C
:101CD0005049EDA2E092007AC5C3E5829400E58305
:101CE000941C5093200010438F02438F0175B7A5B9
:101CF00075B7F1F030001FA827A9280809438F0104
:101D0000538FFDD804D902A11689AAE275B7A5752B
:101D1000B7F1F0A3A103538FFC81757AC1BD030C09
:101D2000E493A3FAB136DCF8B12E81758177AA224B
:101D3000AB23B152EBFAEA6222752608C3E52313FE
:101D4000F523E52213F52250066323A0632201D573
:101D500026EAB1BFB1BF75260AEAF4200102D28596
:101D6000300102C285B1BFC3134002C201D526EBC8
:101D700022B175EAFB208502A175308502A17A7532
:101D80002608AE24AF25C3EF13FFEE13FEB1C3B197
:101D9000BFC3EA133085024480FA30E703632201AF
:101DA000C3E52313F523E52213F52250066323A090
:101DB000632201D526D9E52265236523F52222AECB
:101DC00024AF250E0FDEFEDFFCD20122424C486517
:0A1DD0006C6934373132F33006013C
:00000001FF
